:0400000000000428D0
:080008008A110A120728853055
:10001000831603138600AD2086014220A720831299
:100020000313AD00203A031939282D08613A03194A
:100030002A282D086F3A03192F282D08703A031922
:1000400034282D08713A031D3C28183083120313FD
:1000500086003C2878308312031386003C285830F1
:100060008312031386003C28383083120313860062
:100070003C28831203138601023083120313860681
:100080000E280800B730FF0000307920BE30FF0096
:1000900000307920C530FF0000307920D430FF00D7
:1000A00000307920E030FF0000307920F030FF0090
:1000B00000307920FE30FF000030792008008312E4
:1000C0000313A8007F08A700A90129082707AA0091
:1000D0002808AB000318AB0A2A0884000008AC000B
:1000E000031978282C08992083120313A90A65287C
:1000F000080083120313A2007F08A100A3012308B4
:100100002107A4002208A5000318A50A8B282508AA
:100110008A0024088200872083120313A600260881
:10012000031998282608992083120313A30A7F280D
:10013000080083120313A000831203130C1E9C28D3
:1001400083120313200883120313990008008312FB
:1001500003138C1EA7281A08080081308316031386
:1001600099002430980090308312980008004D3494
:1001700065346E3475340A340D3400342D342D3426
:100180002D342D340A340D34003471342E342D3492
:1001900020346134643465346C3461346E347434C6
:1001A00065340A340D34003461342E342D34203457
:1001B000613474347234613473340A340D3400346D
:1001C0006F342E342D34203469347A3471347534DC
:1001D000693465347234643461340A340D34003463
:1001E00070342E342D3420346434653472346534E4
:1001F0006334683461340A340D3400344534533484
:1002000050344134433449344F342E342D34203467
:10021000503461347234613472340A340D34003431
:02400E00FF3F72
:00000001FF
